:100000000C9463020C9480020C949B020C9480026A
:100010000C9480020C9480020C9480020C94800258
:100020000C9480020C9480020C94E2210C948002C7
:100030000C9480020C9480020C9480020C94800238
:100040000C9480020C9480020C9480020C94800228
:100050000C9480023E063E066A066A06D206FD073A
:10006000FD07FD07F00689079A079A07165C1E0030
:100070001F0020002100220023002400250026006C
:1000800027002D002E00350031002B0014001A002F
:100090000800150017001C0018000C0012001300C7
:1000A0002F0030002A000000E000040016000700C6
:1000B00009000A000B000D000E000F003300340091
:1000C000280000000000E1001D001B0006001900D0
:1000D0000500050011001000360037003800E5006B
:1000E00001510000E300E2002C00E30000000000EA
:1000F0002C00E600E400000000000000000000000A
:10010000000029004B004E0000000000000000002D
:1001100000000000000000000000000000000000DF
:1001200001000100010001000100010001000100C7
:1001300001000100010001000100010001000100B7
:1001400001000100010001000100010001000100A7
:100150000100010052000100010000000100010047
:100160000100010001000100010001000100010087
:1001700050004F00010000000000010001000100DC
:100180000100010001000100010001000100010067
:100190005100010001000000010001000100010008
:1001A000000000000100010001000000000000004C
:1001B000000000000000010001000100000000003C
:1001C000000000000000000000000000000000002F
:1001D0000000000000047F3F1F6432146432147872
:1001E0003C1E1E140A052223252628292A2C2D2FE1
:1001F0003032333536383A3B3D3E4042434547493D
:100200004A4C4E5051535557595A5C5E6062646671
:1002100068696B6D6F71737577797B7D7F8183857D
:1002200087898A8C8E90929496989A9C9E9FA1A37F
:10023000A5A7A8AAACAEAFB1B3B4B6B8B9BBBCBEA3
:10024000BFC1C2C3C5C6C7C9CACBCCCDCED0D1D21F
:10025000D2D3D4D5D6D7D7D8D9D9DADADBDBDBDC21
:10026000DCDCDCDCDDDDDDDDDCDCDCDCDCDBDBDBCD
:10027000DADAD9D9D8D7D7D6D5D4D3D2D2D1D0CE2D
:10028000CDCCCBCAC9C7C6C5C3C2C1BFBEBCBBB932
:10029000B8B6B4B3B1AFAEACAAA8A7A5A3A19F9EB0
:1002A0009C9A98969492908E8C8A89878583817F78
:1002B0007D7B79777573716F6D6B69686664626059
:1002C0005E5C5A5957555351504E4C4A4947454325
:1002D00042403E3D3B3A3836353332302F2D2C2AC2
:1002E000292826252322FFAA7F554000010101016C
:1002F00001010101010202020202020202020303E1
:1003000003030303030304040404040404050505B0
:100310000505060606060607070707070808080872
:10032000090909090A0A0A0B0B0B0C0C0C0D0D0D1F
:100330000E0E0E0F0F0F10101111111212131314B5
:1003400014151516161717181819191A1A1B1B1C2D
:100350001D1D1E1E1F202021222223242425262687
:10036000272829292A2B2C2D2D2E2F3031323233BC
:100370003435363738393A3B3C3D3E3F40414243C5
:100380004445464748494A4C4D4E4F5051535455A9
:100390005658595A5B5D5E5F616264656668696B59
:1003A0006C6D6F7072737577787A7B7D7E808283D7
:1003B0008587888A8C8E8F91939596989A9C9EA01B
:1003C000A2A3A5A7A9ABADAFB1B3B5B7BABCBEC028
:1003D000C2C4C6C9CBCDCFD1D4D6D8DBDDDFE2E4F1
:1003E000E7E9EBEEF0F3F5F8FAFDFF09023B000256
:1003F0000100A0FA09040000010301010009210124
:1004000001000122400007058103080001090401E1
:100410000001030000000921010100012232000750
:100420000583030800011201100100000008A0204C
:100430002E420002010200010C0341006C00690021
:1004400063006500000008035400470052000000EC
:100450000403090405010980A101850319012AB7D4
:1004600000150126B700950175108100C0050C0923
:1004700001A101850419012AA002150126A00295F7
:100480000175108100C005010906A101050719E0E9
:1004900029E7150025019508750181029501750868
:1004A00081030507190029FF150026FF0095067531
:1004B0000881000508190129059505750191029526
:1004C0000175039103C011241FBECFE5D8E0DEBF44
:1004D000CDBF11E0A0E6B0E0ECE5FCE402C0059081
:1004E0000D92A232B107D9F723E0A2E2B1E001C038
:1004F0001D92A832B207E1F70E94F6130C942C2645
:100500000C940000A82FB92F80E090E041E050EA61
:10051000609530E009C02D9182279795879510F05E
:1005200084279527305EC8F36F5FA8F30895EADF4C
:100530008D939D930895CF93CFB7CF93C395839B0E
:10054000E9F7839B0EC0839B0CC0839B0AC0839BEF
:1005500008C0839B06C0C091FF02C395C093FF02F1
:10056000A6C0DF93C091FE02DD27CA5FDC4F839BEC
:1005700002C0DF91E6CF2F930F931F9300B32FEFAD
:1005800003FB20F94F933F9310B34FEF012703FB79
:1005900021F93BE031C04E7F012F10B3216028C00C
:1005A000102F4D7F2260000000B329C04B7F2460D4
:1005B000012F000010B32BC010B3477F28602AC062
:1005C0004F7E00B320612CC04F7D10B320622FC03E
:1005D0004F7B00B3206432C0422700B349934FEFF2
:1005E0000000102713FB20F910B31C70C9F1297FFC
:1005F00091F2012703FB21F900B3237F89F23150E7
:1006000058F1102713FB22F910B3277E79F2012746
:1006100003FB23F92F7C81F200B3102713FB24F98D
:100620002F7971F200C010B3012703FB25F92F7356
:1006300059F200C000B3102713FB26F9223040F214
:1006400000C010B3012703FB27F9243028F64F77A9
:10065000206810B30000F9CF10E81ABF00271CC0B3
:100660003B503195C31BD04010E81ABF0881033CB2
:1006700011F10B3401F12091FB021981110F1213BA
:10068000EDCF4A81441F093669F10D3211F0013E68
:1006900029F74F7009F0042F009304033F914F9105
:1006A0001F910F912F91DF91CAB7C7FD47CFCF910F
:1006B000CFBFCF91189520910403222379F3109195
:1006C0000203112309F044C034300AF443C03093CC
:1006D00002032093FD021091FE023BE0311B309398
:1006E000FE0238C000910203013094F50AE54F7014
:1006F00049F43091840034FD2FC000938400C8ED8C
:10070000D2E02EC0433059F0443091F03091E302F2
:1007100034FD22C00093E302C4EED2E021C0309148
:100720001C0334FD19C000931C03CDE1D3E018C0B5
:100730003091EF0234FD10C00093EF02C0EFD2E021
:100740000FC02795A8F45150A9F4220F0000F9CF4B
:100750004AE503C042ED01C0432FC4E1D0E032E0DE
:1007600011B31C60939A11BB02B320E41CE05F93A9
:10077000012756E002BB279520F4515021F4220FA7
:10078000F9CF012756E000003B5A02BBD0F2279573
:1007900028F4515029F4220F0000F9CF012756E028
:1007A000279502BB20F4515021F4220FF9CF0127E5
:1007B00056E02991332302BB21F6037F10910303F6
:1007C000110FC651D04002BB11F01093FB0210E88C
:1007D0001ABF086011B3137F402F437F5F9100C0A1
:1007E00000C002BB11BB42BB59CF81E0089581E03C
:1007F00008950C94F70308950C94FB031F93CF9373
:10080000DF9300D000D01F92CDB7DEB749835A8363
:100810006B833091250189819A81311114C066233F
:1008200059F0222349F00E94360A182F682F898137
:100830009A810E94DF0903C00E940A0A182F698169
:100840007A81812F04C00E94360A69817A810F90D3
:100850000F900F900F900F90DF91CF911F910C94FC
:100860006411FC01262F4081518162817381848152
:100870000C94FE0381E00895CF93DF93EC0160E0D8
:100880000E943104BE01DF91CF910C94FC030C94C3
:10089000AD120C94A91208950E9489080E944B047D
:1008A0002FEB87E299E0215080409040E1F700C0B3
:1008B00000000C9408220F931F93CF93DF938C01B9
:1008C00061E00E943104EC01B8010E94F903882321
:1008D00009F44BC0B801CE010E94F11B882309F432
:1008E00044C0B801CE010E94C41F8823F1F1B801B1
:1008F000CE010E94F01C8823C1F1B801CE010E94F4
:10090000201F882391F1B801CE010E94351A882357
:1009100061F1F8018281882309F1CB358DE5D80793
:10092000C1F050F4C115FCE5DF0781F0CF3DDC4597
:10093000A9F40E946D0F19C0CC35EDE5DE0761F01A
:10094000CD35DD4559F40E94B00E08C00E944C041C
:100950000CC00E94B90E02C00E94BC0EC801DF91FB
:10096000CF911F910F910C94F50380E0DF91CF910F
:100970001F910F9108950E948C2180E00E94261CF7
:100980000C94F4040E94151B0E94F7040C9492210D
:1009900008950C94C80481E00895CF93C82F0E9455
:1009A000CB04882379F0C0FF02C0909A01C09098D0
:1009B000C1FF02C0919A01C09198C2FF02C0969AED
:1009C00001C09698CF910895889A9098899A9198A5
:1009D0008E9A96980895CF93C82F0E94C9048C2FA1
:1009E0000E94CD04CF91089580E00C94EB040E9406
:1009F000F9200C94EB040E94F920909124018917AE
:100A000021F0809324010C94EB040895CF93DF939D
:100A1000CDB7DEB72B970FB6F894DEBF0FBECDBFB4
:100A20004F83588769877A878B8761110E94FC0DF5
:100A30009E012F5F3F4F86E0F90111928A95E9F7F9
:100A400085E0FE013796D90101900D928A95E1F774
:100A500089819A814C815D81452B31F09F3F31F432
:100A600091E08F3F19F403C091E001C090E090FF46
:100A700009C049815A816B817C818D819E810E9450
:100A80001D0D05C0C9010E943A048111F2CF2B96B9
:100A90000FB6F894DEBF0FBECDBFDF91CF910895A2
:100AA000FC01808191810E94780A0895CF93882368
:100AB00009F44DC0C82F8CEF8C0F813AF8F48C2FBD
:100AC0000E94E41E811143C06C2F809162009091BE
:100AD00063000E944821882349F06C2F80916200B6
:100AE000909163000E9480210E941E0E6C2F8091C5
:100AF0006200909163000E947E210CC080E28C0F06
:100B0000883058F4C77081E001C0880FCA95EAF7B1
:100B10000E94DF0DCF910C941E0EEBE5EC0FE3303D
:100B200040F4F0E0ED54FF4F808190E0CF910C94C1
:100B30001021C85AC73158F4EC2FF0E0EE0FFF1F18
:100B4000EB57FF4F80819181CF910C942621CF915B
:100B50000895882349F1682F8CEF860F813A38F485
:100B600080916200909163000E9480210CC080E21D
:100B7000860F883050F4677081E001C0880F6A9555
:100B8000EAF70E94E50D0C941E0E8BE5860F83306C
:100B900020F480E090E00C941021685A673120F432
:100BA00080E090E00C94262108951F93CF93DF936B
:100BB000182FEB010E945605209741F087EB9BE030
:100BC0000197F1F700C000002197F6CF812FDF9148
:100BD000CF911F910C94A905893319F060E070E062
:100BE00002C060E570E00C94D505882321F00E94D6
:100BF000DF0D0C941E0E0895882321F00E94E50D50
:100C00000C941E0E0895CF92DF92EF92FF920F93F5
:100C10001F93CF93DF937C01D62FC72FFC01128146
:100C2000058102950F700E94D50D8823B9F011231C
:100C3000A9F08C2F807F803421F080E28D0F8830E6
:100C400068F080917F0282FD09C082E00E947E0EE2
:100C50000E94D50D91E0D82ED92601C0D12CCC2EE2
:100C6000C2948FE0C8228C2D90E08C30910508F062
:100C7000C4C1FC01E65DFF4F0C947B258C2F807F67
:100C8000CF70882311F0C295C07F112399F0CC2337
:100C900009F49FC180E28D0F883010F0D11104C09B
:100CA0008C2F0E94DF0D03C08C2F0E94EF0D0E943D
:100CB0001E0E8FC18D2F0E94A905CC2309F49DC162
:100CC00080E28D0F883038F1DD2329F18C2F0E94CE
:100CD000F50D24C08C2F807FCF70803211F0C2952B
:100CE000C07FDD2319F0D130A1F13DC080917F029A
:100CF00082FF17C0112349F0CC2329F08C2F0E94CA
:100D0000DF0D0E941E0E80E065C180E00E94A905F3
:100D1000CC2309F472C18C2F0E94E50D0E941E0E97
:100D20006CC1112371F0002341F0013031F40E94B5
:100D3000FF0D8C2B0E94070E60C10E94FF0D8C2BB3
:100D40001DC0002319F0013009F457C10E94140E90
:100D500025C0112321F0063008F04FC10EC0053028
:100D600008F04BC11BC0112361F0002331F0F701E3
:100D7000858180FF2EC18F7085838C2F0E94F505A1
:100D80003CC1002359F0D93309F034C1FFEF0DEE17
:100D900012E0F15000401040E1F72AC18C2F0E9470
:100DA000FC052BC18C2F86958695837019F08130B8
:100DB00061F023C1112321F08D2F9C2F937002C06D
:100DC00080E090E00E94102120C1112321F08D2F9E
:100DD0009C2F937002C080E090E00E94262115C1F4
:100DE0008C2F837009F047C011110BC12D2F229554
:100DF00026952770220F220F6D2F6F70862F90E09F
:100E0000A0E0B0E0022E04C0880F991FAA1FBB1FEC
:100E10000A94D2F7D4FF10C04FE050E060E070E0D9
:100E200004C0440F551F661F771F2A95D2F74095BF
:100E300050956095709503C040E050E0BA01C695AA
:100E4000C695C3708A019B01082B192B2A2B3B2BBB
:100E5000C901B801C23049F058F4C13019F00E94FC
:100E6000F508CFC00E94E308CCC00E940709C9C0A2
:100E70000E94E108C6C0112319F08C2F817001C0B7
:100E80008695882309F4BDC02D2F229526952770BD
:100E9000220F220F6D2F6F70862F90E0A0E0B0E040
:100EA000022E04C0880F991FAA1FBB1F0A94D2F7F5
:100EB000D4FF10C04FE050E060E070E004C0440F89
:100EC000551F661F771F2A95D2F74095509560955C
:100ED000709503C040E050E0BA01C695C695C37056
:100EE0008A019B01082B192B2A2B3B2BC901B80126
:100EF000C23049F058F4C13019F00E94BA0981C0DB
:100F00000E94A8097EC00E94CC097BC00E941B09D8
:100F100078C0CF70112339F08C2F0E9441098D2F9A
:100F20000E94F5056EC08D2F0E94FC058C2F0E943B
:100F3000620967C0D23F21F128F4D03F41F0D13F90
:100F4000C1F043C0D33F19F1D43F79F03EC0112323
:100F500041F0053008F051C08C2F8F710E94870935
:100F60004CC0063008F049C0F7CF80917F0282FF65
:100F700018C0112339F08C2F8F710E9441093DC098
:100F80001123C9F38C2F8F710E94620936C011237F
:100F900029F08C2F8F710E942C092FC00E942709E5
:100FA0002CC0112349F0CF718C2F0E94410963E0BE
:100FB0008C2F0E94630E21C081E00E947E0E0230C1
:100FC000E0F082E00E947E0E18C0112331F0002371
:100FD00091F28D2F0E94560510C0002399F2D9334B
:100FE00049F41FEF2DEE32E0115020403040E1F780
:100FF00000C000008D2F0E94A90588EF8C0D843061
:1010000020F40E94F9200E94EB04DD20C9F00E9428
:10101000D10D80FD15C0F70112820E94CB0D0E94F8
:101020004109C7010E9441080E94CB0DDF91CF9179
:101030001F910F91FF90EF90DF90CF900C94620979
:10104000DF91CF911F910F91FF90EF90DF90CF90A4
:1010500008950F931F93CF93DF93EC0168817981FB
:101060008A810E94830A8C010E94DE090E94CF08B7
:10107000B801CE010E940306DF91CF911F910F911D
:101080000895CF93DF93EC01988189812B813C8176
:10109000232B31F08F3F31F481E09F3F19F403C0DF
:1010A00081E001C080E080FD1DC0CE010E945B0494
:1010B000811110C00E94D50D8823A1F08A81882358
:1010C00089F080917F0282FD0DC082E0DF91CF9197
:1010D0000C947E0ECE010E942908CE01DF91CF91A3
:1010E0000C943C04DF91CF91089580E090E00E9441
:1010F000102180E090E00E9426210E94FC0D0C94BB
:101100001E0E80916200909163000E9482210C94D7
:1011100075080E94EC0D0C94810892959F70963092
:1011200079F010F4925001C09A50923068F4803FE8
:1011300069F018F4883E40F409C0843F29F406C0E1
:10114000883E20F0813F11F080E0089581E008950D
:10115000FC01808191810E94780A0E948D08089587
:10116000CF93DF9300D000D01F92CDB7DEB70F90A2
:101170000F900F900F900F90DF91CF910895CF9324
:10118000DF9300D000D000D0CDB7DEB726960FB6E3
:10119000F894DEBF0FBECDBFDF91CF9108950895C3
:1011A00008950C94D0080C94D1080E94D308609341
:1011B00066017093670180936801909369010C94B4
:1011C00075080C94D5080F931F9300916601109138
:1011D00067012091680130916901602B712B822B8E
:1011E000932B1F910F910C94D5080F931F9300918F
:1011F00066011091670120916801309169016023B7
:101200007123822393231F910F910C94D5080F9380
:101210001F93009166011091670120916801309140
:10122000690160277127822793271F910F910C94E2
:10123000D5080C94D0080E9419096093620170933C
:10124000630180936401909365010C94750860E0DC
:1012500070E0CB010C941B090F931F9341E050E009
:1012600060E070E08A019B0104C0000F111F221F83
:10127000331F8A95D2F7C901B8011F910F910C94C1
:101280001B090F931F9341E050E060E070E004C041
:10129000440F551F661F771F8A95D2F78091620110
:1012A00090916301A0916401B09165018A019B0155
:1012B000082B192B2A2B3B2BC901B8011F910F9129
:1012C0000C941B090F931F9341E050E060E070E025
:1012D00004C0440F551F661F771F8A95D2F74095AB
:1012E0005095609570958091620190916301A091F5
:1012F0006401B09165018A019B01082319232A2307
:101300003B23C901B8011F910F910C941B090F9346
:101310001F9341E050E060E070E004C0440F551FAF
:10132000661F771F8A95D2F78091620190916301C1
:10133000A0916401B09165018A019B0108271927DA
:101340002A273B27C901B8011F910F910C941B0953
:101350000F931F930091620110916301209164012A
:1013600030916501602B712B822B932B1F910F9174
:101370000C941B090F931F9300916201109163015C
:1013800020916401309165016023712382239323AE
:101390001F910F910C941B090F931F9300916201F1
:1013A00010916301209164013091650160277127DC
:1013B000822793271F910F910C941B0908952FE00A
:1013C000929F800D1124E82FE695E695E6958770AB
:1013D00051E001C0550F8A95EAF785E0E89FF001DA
:1013E0001124EA5DFE4F20E030E070E04081CB0147
:1013F000022E02C0969587950A94E2F78170819536
:1014000084278523842781932F5F3F4F2530310523
:1014100069F708952FE0929F800D1124682F66953B
:1014200066956695982F977085E0689FB0011124A6
:1014300040E050E080E0FB01E40FF51FEA5DFE4F65
:10144000208130E0092E02C0369527950A94E2F7F4
:1014500021703327042E01C0220F0A94EAF7822B51
:101460004F5F5F4F4530510531F70895BF92CF92DE
:10147000DF92EF92FF920F931F93CF93DF938C0134
:10148000C0906201D0906301E0906401F09065012A
:101490008091660190916701A0916801B091690106
:1014A000C82AD92AEA2AFB2ACFE1D0E0D701C6010F
:1014B0000C2E04C0B695A795979587950A94D2F7F8
:1014C00080FD04C0219790F7B12C07C0BC2EB80155
:1014D0008C2F0E9477110197A9F38B2DDF91CF916B
:1014E0001F910F91FF90EF90DF90CF90BF900895E4
:1014F000CF93DF93EC010E94360ABE010E94771160
:10150000DF91CF9108951F93CF93DF93EB019091DB
:101510002501992321F0CB010E94780A13C088236A
:1015200049F0CB010E94360A182F682FCE010E9485
:10153000DF0904C0CB010E940A0A182FBE01812FC7
:101540000E947711DF91CF911F9108951F93CF9340
:10155000DF93C0916A0116E080916B01C81799F082
:10156000D0E01C9FF0011D9FF00D1124E459FE4FA7
:101570004081518162817381848195810E94BF087D
:101580002196C770E9CFDF91CF911F9108954091C7
:101590009C0150919D0160919E0170919F018091ED
:1015A000A0019091A1010C94BF08EF92FF920F93BC
:1015B0001F93CF93DF938091A10182958F7009F0E3
:1015C00065C080919E01882309F460C080916A0102
:1015D000F0906B0110919C0100919D0160919F0121
:1015E0007091A00191E01F3F09F090E0C091600070
:1015F000D0916100292F96E0E92E8F1509F446C09D
:101600006115710521F00F3F21F030E003C031E09A
:1016100001C0322F90E030FD36C0E89EF001E99E17
:10162000F00D1124DF01A459BE4F11963C91119782
:10163000301329C03C91311326C012963C91129769
:10164000311121C013964D915C911497461B570B95
:101650004C175D07C0F48091A1018F708061809369
:10166000A101EF58FE4F80818F70806180838CE9EB
:1016700091E00E944108DF91CF911F910F91FF905F
:10168000EF900C94A60A01968770B7CFDF91CF91A7
:101690001F910F91FF90EF9008959F92AF92BF928C
:1016A000CF92DF92EF92FF920F931F93CF93DF932E
:1016B000CDB7DEB761970FB6F894DEBF0FBECDBFD2
:1016C0008C0185E0F801DE011D9601900D928A954E
:1016D000E1F7D8011296EC9090919C01E0919D0168
:1016E00020919F013091A0012115310531F0EF3F8C
:1016F00031F481E09F3F19F403C081E001C080E034
:10170000B82FB1709B2E80FD47C1D8014C91119626
:101710005C9111971396AD90BC9014978CE9C82EEC
:1017200081E0D82EF0909E01B501621B730B2091D1
:10173000600030916100FF2009F4D9C08091A101BF
:101740006217730708F095C0282F207F09F052C058
:101750005E1313C0491311C0FE2CE1100EC08F7030
:1017600080618093A1010E94C70AC6010E944108BE
:101770008091A101F80185834DC1AB2831F05F3F15
:1017800031F481E04F3F19F403C081E001C080E0F3
:1017900080FD03C081E08E2502C080E090E0F82F3C
:1017A000F170FF2E80FF1CC080916A0120916B01B7
:1017B00036E0821709F40BC190E0389FF001399FA1
:1017C000F00D1124E459FE4F6181561306C060816B
:1017D000461303C06281E61203C001968770E9CF09
:1017E000FE2CEE2009F416C18091A1018160809346
:1017F000A10154C05E1306C0491304C0E11002C029
:10180000F80199C0C8010E94A808882361F1EE2060
:1018100051F12091A101822F82958F7090E0029763
:1018200074F080919C0190919D0198878F83198617
:10183000BB86AA862C87CE0107960E94410886E0C7
:10184000F801ACE9B1E001900D928A95E1F70E94B0
:10185000D50A0E94C70A0AC05E1711F1C8010E948A
:10186000A80881112CC0C8010E944108FF24F394EC
:10187000D1C0282F207F81F77A2DB98AA88A6E2DB2
:1018800089890E94B0088CE991E00E94410886E0B5
:10189000D6011D928A95E9F70E94C70AF12CBAC0B9
:1018A0004913DCCFE110DACFF8018583C8010E942B
:1018B000410886E0D6011D928A95E9F7ABC0EE207B
:1018C00091F22091A101822F82958F7090E0029772
:1018D0000CF4B5CF80919C0190919D019A838983EE
:1018E0001B82BD82AC822E83CE010196A6CF6217E9
:1018F000730708F044C0FE2CEE2009F4B4CF5E1349
:1019000030C049132EC02091A10120FD21C0822F9B
:1019100082958F70482F50E041155105C9F0F801AC
:1019200025834F30510541F08F5F982F9295907F1E
:10193000822F8F70892B8583C8010E94410886E021
:10194000F801ACE9B1E001900D928A95E1F73CC055
:1019500086E0F801ACE9B1E001900D928A95E1F7DB
:1019600059C0C8010E94A808811169CF8091A101C6
:1019700081608093A101C8010E9441084BC07A2D6B
:10198000B98AA88A6E2D89890E94B00886E0D6019E
:101990001D928A95E9F718C0EE2009F464CFC801BA
:1019A0000E94A808F82E882309F45DCF86E0F8018C
:1019B000ACE9B1E001900D928A95E1F78CE991E0F4
:1019C0000E9450050E94D50A0E94C70A23C04D8775
:1019D0005E878D859E850E94780A292F22952F701B
:1019E000223028F49F7039F0811105C00BC02430DB
:1019F00028F49F7049F4805E883020F0C8010E946E
:101A000041089F2CF92C06C0D80115969C91907F17
:101A100091F7F8CF8F2D61960FB6F894DEBF0FBE09
:101A2000CDBFDF91CF911F910F91FF90EF90DF908D
:101A3000CF90BF90AF909F9008951F93CF93DF9367
:101A4000CDB7DEB72C970FB6F894DEBF0FBECDBF73
:101A50004F83588769877A878B879C87CE01079643
:101A60000E944D0B8823D1F09F8188852A853B8574
:101A7000232B31F08F3F31F481E09F3F19F403C0F5
:101A800081E001C080E080FD47C04F8158856985B5
:101A90007A858B859C850E94BF083EC086E0FE014A
:101AA0003796DE01119601900D928A95E1F7FF813C
:101AB000E8856A857B856115710531F0EF3F31F46A
:101AC00081E0FF3F19F403C081E001C080E080FDA8
:101AD00023C020916B0130E0C901019687709927DE
:101AE00040916A0150E084179507F1F1F983EA8388
:101AF0007D836C8396E0929FD001939FB00D11245B
:101B0000A459BE4FFE01319601900D929A95E1F7CE
:101B100080936B010E94A60A16E080916A01909161
:101B20006B01891771F1189FC001112484599E4FD0
:101B30000E944D0B882329F1E0916A011E9FF0015C
:101B40001124E459FE4F4081518162817381848167
:101B500095810E94BF0880916A0190E0019687708C
:101B6000992780936A01D9CF0E94890810926B014E
:101B700010926A01ECE9F1E086E0DF011D928A959E
:101B8000E9F72C960FB6F894DEBF0FBECDBFDF91FC
:101B9000CF911F9108958091AA018595859585958E
:101BA00008958091AA01877008959091AA01977075
:101BB00081E009F480E008958091B5010895909145
:101BC000B501892B8093B501089580959091B50159
:101BD00089238093B50108951092B50108959091DD
:101BE000B401892B8093B401089580959091B4013C
:101BF00089238093B40108951092B40108958091CF
:101C0000AB01089508950C94020E0C94030E90916C
:101C10007F0292FD08C09091AB01981721F080934C
:101C2000AB010C94050E08958091AB01882329F037
:101C30001092AB0180E00C94050E0895CF93DF93D2
:101C4000E0916200F09163008091B5018083E091A2
:101C50006200F091630090818091B401892B8083B0
:101C60008091AB01882381F0E0916200F0916300E4
:101C70009081892B808380916200909163000E9403
:101C80003C2181110E94140EC0916200D09163002A
:101C900048E050E062EA71E0CE010E94CB25892B3A
:101CA00069F088E0FE01A2EAB1E001900D928A9508
:101CB000E1F7CE01DF91CF910C940521DF91CF9117
:101CC00008950C94020E90917F0292FD10C098E04E
:101CD000899F90011124262B2093AA010E9441097B
:101CE0008091AA018595859585950C94610E0C943B
:101CF00041091092AA0180E00C94610E2091AA0182
:101D0000809582238093AA01982F977099F430E0F0
:101D1000482F082E000C550B2417350759F09091C9
:101D20007F0292FD07C08595859585950E94620981
:101D30000C94790E089590917F0292FB222720F94E
:101D4000281769F080FB92F990937F0280917E02C0
:101D500090917F020E94E90E82E00C947E0E08951D
:101D600080917F0282FB882780F991E089270C947B
:101D70009B0E81E00C949B0E80E00C949B0E6FEF09
:101D80007FEF80E090E00C94092680E090E00E94D4
:101D9000E62521E0893E9E4F09F020E0822F08953C
:101DA00082E090E00C94D82583E090E00C94D82554
:101DB000CF9384E090E00E94D825C82F82E290E083
:101DC0000E94D8252C2F30E0A901582BCA01CF91B1
:101DD0000895CF93C92F682F84E090E00E94EC25EE
:101DE0006C2F82E290E0CF910C94EC25AB01BC010A
:101DF0008FE090E00C94FD25AB01BC0183E190E005
:101E00000C94FD2560E070E0CB010C94FC0E60E0CA
:101E100070E0CB010E94F60E0C94020F69EE7EEF8B
:101E200080E090E00E94092660E082E090E00E945D
:101E3000EC2560E083E090E00E94EC2510926601C2
:101E400010926701109268011092690160E084E0CD
:101E500090E00E94EC2560E082E290E00E94EC2598
:101E600060E085E090E00E94EC2560E086E090E094
:101E70000E94EC256FEF87E090E00E94EC2540E0A7
:101E800050E0BA0188E090E00E94FD2560E08DE01E
:101E900090E00E94EC2540E050E0BA0188E190E03B
:101EA0000E94FD2560E087E190E00E94EC2540E083
:101EB00050E0BA018CE190E00E94FD2560E070E006
:101EC00080E290E00E94092640E050E0BA0188E1FB
:101ED00090E00E94FD250C94070F0C940E0F682FC4
:101EE0008EE090E00C94EC250E94C7216093C6011F
:101EF0007093C7018093C8019093C9016093C20198
:101F00007093C3018093C4019093C501089584B771
:101F1000806884BF84B7806884BF089581E0089595
:101F20000C948E0F08950C94920F0C94920F0C94B5
:101F3000950F0C94920F0C94990F0C94920F0E9491
:101F4000870F83E592E10E94EF200E949D0F0C9481
:101F50009B0F0E94930F0C94920F0E9470120E948C
:101F6000E4040C94C61C0E94B4210E9455130E94E4
:101F7000AD0F0E94151B0E9454190C94970F5F928D
:101F80006F927F928F929F92AF92BF92CF92DF9289
:101F9000EF92FF920F931F93CF93DF93CDB7DEB7EE
:101FA0002A970FB6F894DEBF0FBECDBF0E946A130A
:101FB000C82E81110E94740F36EB832E31E0932ED0
:101FC00000E010E0502E802F0E9494125C01F4017A
:101FD000619071904F016826792661147104B1F403
:101FE0000F5F1F4F0630110569F78FEF89838A83D2
:101FF0001B820E94BB218160782F9D838C83498145
:102000005A816B818D810E9406053AC08091CA0178
:1020100081FD0E949D12D12CEE24E394F12CC3018A
:102020008E219F21892B29F10E94900F8823A9F0EE
:10203000DE825F82AE20BF2081E0AB2809F480E021
:1020400088870E94BB218160782F9A8789874E817B
:102050005F8168858A850E940605000F111FF801BF
:10206000EA54FE4F80819181E826F926F182E082D0
:1020700007C0D394EE0CFF1CFFE0DF12D0CFB0CF2F
:1020800081E0C11001C080E02A960FB6F894DEBF4F
:102090000FBECDBFDF91CF911F910F91FF90EF90B9
:1020A000DF90CF90BF90AF909F908F907F906F9078
:1020B0005F9008950E94BF0F0E9487190E94C51C5F
:1020C0000C94FB04CF93DF930E947C11EC018115EB
:1020D00022E59207E8F5811531E5930708F0B6C0CF
:1020E000883E910528F5803E910508F0E9C0883AC0
:1020F000910570F4853A910508F07AC08130910518
:1021000009F473C008F4D9C0049708F0D9C0D5C049
:102110008F3B910508F0D1C0C85AD0E0CC0FDD1F2D
:10212000CA54DF4F0990D881C02DCE019464C9C034
:10213000811540E5940708F069C0811550E49507C2
:1021400008F060C09A9581159F4108F4B9C0B5C0E8
:10215000811536E5930728F5811545E5940708F0C4
:1021600092C0811554E5950708F087C0AC01437013
:102170005527282F26952695C115D34508F06CC004
:1021800081E090E002C0880F991F4A95E2F740E293
:10219000249F90011124EC01C22BD32BCE019C680B
:1021A00090C081152AE5920780F4811539E59307DF
:1021B00008F072C0811548E5940708F47EC0D82F56
:1021C000CC27CE01806F906A7CC0905681159042DA
:1021D00008F073C08D2F8F710E941012DD27D0621E
:1021E0008F71AE01582BCA016CC081E090E069C0CC
:1021F000C55AD0E0CC51DF4F8881C82FD0E0CE0146
:1022000090645FC0DF70CE01906A5BC074E0969509
:1022100087957A95E1F7282F23703C2F337081E062
:1022200090E002C0880F991F3A95E2F79C68AC01D4
:10223000522B9A019C2F9F709695969550E2959FF0
:10224000E0011124C9018C2B9D2B3BC0D82FCC273A
:10225000CE01816F906A35C081E090E002C0880FA6
:10226000991F4A95E2F750E2259F90011124EC0155
:10227000C22BD32BCE019A6824C0D82FCC27CE01F5
:10228000846F906A1EC00E9410128F7190E0D82F48
:10229000CC27CE01906215C08F700E94101294E07E
:1022A000D695C7959A95E1F7CF70D0E0DC2FCC2773
:1022B000D0699E01282BC90104C080E090E001C0D4
:1022C000CE01DF91CF9108952AE5829FC0011124AC
:1022D000FC012FE0729FE00DF11D1124E60FF11DAE
:1022E000EE0FFF1FE459FF4F8591949108950E94CE
:1022F00064110E94621008958238910569F1B0F46A
:102300008133910509F46DC048F48932910509F4CF
:1023100063C08A32910509F469C008958533910537
:1023200009F455C089339105B9F00895833E9105AC
:1023300069F138F4803E9105B1F0823E910509F1D2
:102340000895863E9105A9F1873E9105B9F1843E35
:10235000910509F064C023C020917E0220FD4FC08A
:1023600021FD4DC0089580917E0280FD44C0809182
:102370007F0280FF44C080917E0284FD42C083EED4
:102380004DC080917E0282FF38C0F5CF80917E02E1
:1023900082FD33C080917F0280FD31C0ECCF8091FF
:1023A0007F0281FF32C080917E0284FD2AC087EEC9
:1023B00035C080917E0283FF26C0F5CF80917E02DA
:1023C00083FD21C080917F0281FD1FC0ECCF8091F1
:1023D0007E0285FD1CC01DC080917E0285FD19C056
:1023E00016C080917E0286FD16C017C080917E02C5
:1023F00086FD13C010C089E311C082EE0FC080EECD
:102400000DC080E00BC086EE09C084EE07C089E2F3
:1024100005C085E303C08AE201C081E390E008952E
:1024200090917E0292FF0DC0282F2871283019F458
:10243000877F846006C0282F2471243011F48B7F9D
:10244000886093FF0DC0282F2871283119F4877EEA
:10245000846106C0282F2471243111F48B7E886199
:1024600020917F0220FF0DC0382F3871383019F4C9
:10247000877F816006C0382F3171313011F48E7F33
:10248000886021FF0DC0282F2871283119F4877E1C
:10249000816106C0282F2171213111F48E7E88615F
:1024A00094FD877E089580E008950C94BF0E0E94ED
:1024B0006A132FE389E191E0215080409040E1F7D9
:1024C00000C000000E946A1380E00E94941280FF06
:1024D00004C00E9455120C94082208950C945712BF
:1024E0000E94C50E811102C00E946D0F0E94D00E85
:1024F0008093CA010E94D80E90937F0280937E023F
:102500000E946E120E94D40E682F70E080E090E06E
:102510000E94E10860916201709163018091640101
:10252000909165010C941909E82FF0E0EE0FFF1F60
:10253000E457FD4F808191810895089588E78A9539
:10254000F1F7089500C008950C949E1208950C941C
:10255000A6120C94A7120C94A6120C94AB12F89429
:10256000E82FE295EF70F0E031A9282F2F7081E07D
:1025700090E001C0880F2A95EAF7982F9095932351
:1025800091AB92A9892B82AB789408950F931F93F6
:10259000CF93DF93C6EFD0E089918F3F11F00E9477
:1025A000AF1280E0CC3FD807B9F7C7EED0E006EF16
:1025B00010E089918F3F11F00E94AF120C171D0798
:1025C000C1F7DF91CF911F910F910895BF92CF92E4
:1025D000DF92EF92FF920F931F93CF93DF938C01C3
:1025E000C62FD0E0CE018A509F4F6C01FC01908134
:1025F0009F3F09F450C0B62EF894E92FE295EF7092
:10260000F0E081A99F7021E030E001C0220F9A958F
:10261000EAF7822B81AB82A92095282322AB7894FC
:102620000E94A212E7EEF0E046EF50E021E030E039
:10263000E12CF12C61916F3F89F0A62FA295AF702C
:10264000B0E0D0968C9190E06F7002C09595879520
:102650006A95E2F780FD02C0C90102C080E090E007
:10266000E82AF92A220F331F4E175F0719F7F601E0
:1026700080818F3F11F00E94AF1261E0E114F104FC
:1026800009F460E08B2D0E94A412CC0FDD1FC00F57
:10269000D11FF982E882DF91CF911F910F91FF90B6
:1026A000EF90DF90CF90BF9008950E94C6128CE00B
:1026B000ECE8F2E0DF01982F1D929A95E9F7E0E847
:1026C000F2E0DF011D928A95E9F786E00E94B513DA
:1026D0000C944704FF920F931F93CF93DF93CDB7D2
:1026E000DEB72C970FB6F894DEBF0FBECDBF8E01BC
:1026F0000F5F1F4F8CE0F80111928A95E9F7F12CDA
:102700006F2DC8010E94E612F394F6E0FF12F8CF95
:102710004CE050E0B80180E892E00E94CB25FF2415
:10272000F394009709F4F12C892B41F08CE0F80127
:10273000A0E8B2E001900D928A95E1F72F2D46E0D6
:102740006CE872E080E892E00E94B6130E944904AF
:102750008F2D2C960FB6F894DEBF0FBECDBFDF9144
:10276000CF911F910F91FF9008950895FF920F93BD
:102770001F93CF93DF93F82E092F162FD72FC42F37
:10278000222349F081E08093CD010E94BB219093E8
:10279000CC018093CB018091CD018823D9F0809129
:1027A000CB019091CC010E94D321059798F0EF2D99
:1027B000F02FA12FBD2F80E090E04C2F50E0841728
:1027C000950734F4219131912D933D930196F7CFE4
:1027D0001092CD01DF91CF911F910F91FF9008953D
:1027E0000E941D220E94B30F0C942E220E94A92148
:1027F0000E9416220E949F0F0E94F0130E943C220A
:102800000E94A90FFBCFEF92FF920F931F93CF93DC
:10281000DF938B01682F11110AC0442329F0E82FA0
:10282000F0E0E551FD4F6491762F862F75C0212F82
:1028300030E0E82FF0E0442321F0E551FD4FE49132
:10284000F0E046E0049FC0011124CFEFD0E0BE01CC
:102850000E9431254BEA4603C001479F900D112489
:10286000800F911D800F911D982F990F890FAE0138
:10287000421B530B4E9FD0014F9FB00D5E9FB00D7A
:1028800011249B2F189FA0011124452F55278E013D
:10289000041B150B0E9FA0010F9F500D1E9F500D86
:1028A00011247E01E81AF108E29E8001E39E100DDA
:1028B000F29E100D1124212F3327C21BD30BCE9F64
:1028C0009001CF9F300DDE9F300D112462307105D5
:1028D000A9F048F46115710569F061307105C9F41A
:1028E0008B2F752F0DC06430710581F058F0663064
:1028F000710579F47E2F8B2F932F0DC0832F7B2FA3
:102900009E2F09C08E2F7B2F952F05C08E2F732FE2
:1029100002C07E2F852F692FDF91CF911F910F91DC
:10292000FF90EF90089541E00E94031408950895E8
:102930000E9493140895CF93DF93762FE901682FB7
:10294000842F0E949814798368838A83DF91CF91C2
:10295000089580919802282F269530E021153105A1
:1029600019F48170826005C02532310524F0817030
:10297000886480939802089588E090E00C94E025A4
:10298000CF92DF92EF92FF926B017C010E94A9141B
:10299000B701A60188E090E0FF90EF90DF90CF9024
:1029A0000C94FD25E8E9F2E083E0808311828FEF4B
:1029B00082838383148260817181828193810C94EC
:1029C000C0148091980280FF02C08695089580E02F
:1029D000089590919C02933018F49F5F90939C020D
:1029E000882351F0609198027091990280919A0227
:1029F00090919B020C94C014089581E00C94E9140A
:102A000090919C02992319F0915090939C028823F5
:102A100051F0609198027091990280919A02909180
:102A20009B020C94C014089581E00C94001570E092
:102A30000C94D21C609168008091980280FF0AC0BB
:102A40008091670023E0829FC001112483569D4F2F
:102A50000C9417158091690090916A00891780F78E
:102A6000E82FF0E09F01220F331FE20FF31FE35620
:102A7000FD4F1182108212828F5FF0CF90919802E9
:102A800090FF16C09091690020916A00921770F42F
:102A9000E92FF0E0DF01AA0FBB1FEA0FFB1FE3568F
:102AA000FD4F8183608342839F5FF0CF0C941A15A2
:102AB0000895CF93DF9300D01F92CDB7DEB79091EA
:102AC000980290FF0AC09E012F5F3F4F0E949B1407
:102AD0004B8169818A810E943E150F900F900F9063
:102AE000DF91CF910895CF93DF93EC01EC81F0E07B
:102AF000EA51FE4F4491E8E9F2E0628181810E944F
:102B000059158C818F5F8C83DF91CF910895CF937E
:102B1000DF93EC01E8E9F2E0438162818C810E945D
:102B200059158C818F5F8C83DF91CF9108950F931E
:102B30001F93CF93DF9300D01F92CDB7DEB78C01E8
:102B40008091CE0181110AC09E012F5F3F4F4FEF50
:102B50006FEF0E949B148A818093CE01F8018481DB
:102B6000813051F028F0823061F44091CE010AC0EA
:102B70008091CE0140E007C06091CE0140E080E04E
:102B800003C040E080E060E00E943E15F8018481CF
:102B900090E0019663E070E00E94452584830F90E9
:102BA0000F900F90DF91CF911F910F910895AF92E9
:102BB000BF92CF92DF92EF92FF920F931F93CF932A
:102BC000DF9300D01F92CDB7DEB7182FF62E042F5B
:102BD000E22E9091980290FF6DC0E92FE695AE2FFE
:102BE000B0E0A450BF4F8C918093D8019E7F92306B
:102BF00061F49E012F5F3F4F812F0E949B144B81F8
:102C000069818A810E943E1543C0823019F4009187
:102C10009B023EC0863019F41091990239C0893068
:102C2000D9F38931A9F5E9518E2F8170D82EE69517
:102C3000F0E0EA51FD4FA590B490C12CBB24609107
:102C40006B00C61618F52C2D30E0A29EC001A39E85
:102C5000900DB29E900D112470E00E943125812FBD
:102C6000D11002C0860F01C0861B90916900290F08
:102C7000311DA901440F551F240F351F23563D4F09
:102C8000402F6F2D0E949B14C394D9CF0E941A1518
:102C900010939902F0929A0200939B02EE2051F059
:102CA000609198027091990280919A0290919B0292
:102CB0000E94C0140F900F900F90DF91CF911F9141
:102CC0000F91FF90EF90DF90CF90BF90AF9008955D
:102CD000E8E9F2E09181282F4381628188E0890F41
:102CE0000C94D71581E00C946816E8E9F2E0918124
:102CF000282F4381628188EF890F0C94D71581E0DA
:102D00000C947516E8E9F2E0628121E1620F08F4A3
:102D10006FEF282F438181810C94D71581E00C94AB
:102D20008216E8E9F2E0628121E1621B08F460E0CA
:102D3000282F438181810C94D71581E00C94911642
:102D4000E8E9F2E0438121E1420F08F44FEF282F38
:102D5000628181810C94D71581E00C94A016E8E97A
:102D6000F2E0438121E1421B08F440E0282F628118
:102D700081810C94D71581E00C94AF1620E00C945F
:102D8000D715FF920F931F93CF93DF93EC01F12C94
:102D90000FEF10E060916B00F616F0F4809169007F
:102DA0002F2D30E0280F311DC901880F991F280FE2
:102DB000391F23563D4F70E0C8010E944525962FCC
:102DC0008C8140919B0260919A02F99E800D1124A2
:102DD0000E949B14F394DECF0E941A159A818C8175
:102DE00090FF02C08F5F01C081508C83DF91CF9133
:102DF0001F910F91FF900895AF92BF92CF92DF92F3
:102E0000EF92FF920F931F93CF93DF93FC01828188
:102E100080FF02C00FEF01C001E010E042E1A42EEC
:102E200080916B00181708F043C080916900C12E93
:102E3000D12CE601C80FD11DCE01880F991FC80FF4
:102E4000D91FC356DD4F198218821A8234E0E32E4F
:102E5000F12CB12C8091D0018B0D83312CF06A2D97
:102E60000E942325892F05C087FF03C090916B0026
:102E7000890F082E000C990BC816D90691F4809181
:102E80009B028E9DA0018F9D500D11245595479555
:102E9000559547959E0160919A02809199020E94F2
:102EA0009B14B00EF1E0EF1AF108A1F61F5FB8CF46
:102EB0000E941A158091D001013031F4811102C0B5
:102EC00080916B00815007C090E0019660916B008B
:102ED00070E00E9445258093D001DF91CF911F9132
:102EE0000F91FF90EF90DF90CF90BF90AF9008953B
:102EF000CF938091690090916A00891770F4E82F50
:102F0000F0E09F01220F331FE20FF31FE356FD4F46
:102F10001182108212828F5FF0CFC0E060916B004F
:102F2000C617C0F5EC2FF0E070E0CF010E944525F8
:102F300020916900820F2091CF01022E000C330BEB
:102F400090E0E217F307CCF020916600022E000C0F
:102F5000330B2E173F078CF09C01220F331F820F7B
:102F6000931F9C0123563D4F40919B0260919A0212
:102F7000809199020E949B140BC0FC01EE0FFF1F71
:102F80008E0F9F1FFC01E356FD4F118210821282AB
:102F9000CF5FC4CF0E941A15209165008091CF01A8
:102FA000820F8093CF0190916600920F90936600FC
:102FB00019165CF4082E000C990B40916B0050E040
:102FC00041505109841795071CF021952093650005
:102FD000CF9108958F929F92AF92BF92CF92DF923E
:102FE000EF92FF920F931F93CF93DF938C01FC011D
:102FF0004481C42FD0E09E01DE010E9489259B01FF
:10300000AC010E949F256B017C01E0E2F0E0EC1B2B
:10301000FD0BA5E5B0E09B01AC010E949F254B0193
:103020005C019F01DF010E9481259B01AC010E9490
:10303000AA259B01AC012C0D3D1D4E1D5F1DC50138
:10304000B4010E945925C22FD22F2A3228F4F3E06E
:103050002F9F900111240DC025E530E02C1B310974
:10306000C901880F991F280F391F37FF02C02F5F32
:103070003F4F35952795C22FC095F12C85E5E82E59
:10308000ED1A80916B00F816C8F4F1FC02C08E2D89
:1030900001C08D2F909169002F2D30E0290F311D37
:1030A000A901440F551F240F351F23563D4F4C2FA8
:1030B00060919A020E949B14F394E3CF0E941A1528
:1030C000F8018481811102C091E003C0803219F4BB
:1030D0009FEF9093640090916400890FF8018483BE
:1030E000DF91CF911F910F91FF90EF90DF90CF90E4
:1030F000BF90AF909F908F9008950F931F93CF93A1
:10310000DF93EC0100E010E080916B00282F30E0AD
:103110000217130724F5909169009801290F311DBA
:10312000A901440F551F240F351F23563D4F869587
:1031300090E04C81081719071CF4442331F002C0B9
:10314000411103C040919B0201C040E060919A028E
:10315000809199020E949B140F5F1F4FD5CF0E9450
:103160001A158C8190E00196817099278C83DF91EC
:10317000CF911F910F910895E8E9F2E080818E7F51
:10318000808360817181828193810E94C01410923A
:10319000D9012FEB84ED91E0215080409040E1F780
:1031A00000C000000C941A1560919802669570E0BA
:1031B0004BE050E08CE690E00E94BE25892B19F48C
:1031C00081E08093D9010E94BB219093D20180932A
:1031D000D10108959091980290FF35C091708111AE
:1031E00002C0926006C0853210F0986402C0880F59
:1031F000982B90939802662351F0609198027091F9
:10320000990280919A0290919B020E94C014609151
:103210009802669570E04BE050E08CE690E00E94EA
:10322000BE25892B19F01092D90102C00E94D41832
:1032300081E08093D40140919B0260919A02809139
:1032400099020C94BE160895682F90919802969555
:1032500081E0890F853208F081E00C94EA1881E062
:103260000C942419682F9091980296958FEF890FEE
:1032700009F484E20C94EA1881E00C94321961E0BC
:103280000C94EA18E8E9F2E08081816080838695F9
:103290000C943F198091980280FD0C94BC180C94FA
:1032A000421960E00C94EA188091D70181112EC078
:1032B0000E94C50E811104C00E946D0F0E94D2149D
:1032C0000E94BC14609398027093990280939A02B2
:1032D00090939B026E7F61F40E94D2140E94BC14F2
:1032E000609398027093990280939A0290939B0244
:1032F0000E94A9141092D9018091980280FF03C006
:1033000086950E94511981E08093D70108950F930B
:103310001F93CF93DF938091D901882309F485C04F
:103320008091D801E0919802E695E81BE093D301E3
:10333000823049F4F0E0EE51FE4FE491CE2FD0E020
:1033400003E715E149C0863049F4F0E0E152FE4F51
:10335000E491CE2FD0E007E815E13EC0893051F46A
:10336000E695F0E0E452FE4FE491CE2FD0E001EC80
:1033700016E132C08F3051F4E695F0E0E752FE4F8F
:10338000E491CE2FD0E00CEF16E126C0853149F450
:10339000F0E0EA52FE4FE491CE2FD0E008E717E1CB
:1033A0001BC0883181F0833239F4E4EDF1E0C5913E
:1033B000D49107E915E110C0843251F4C4EFD1E093
:1033C0000DE718E109C0C8E2D0E00AEE17E104C039
:1033D000C0EDD7E007E914E18091D401882361F0C2
:1033E0001092D4010E94BB219093D2018093D1010D
:1033F0001092D6011092D5010E94BB21E091D1011B
:10340000F091D2018E1B9F0B8F3F9F4770F4EC0F02
:10341000FD1FF093D201E093D10181ED91E0F8011D
:10342000DF91CF911F910F910994DF91CF911F915F
:103430000F910895882311F0FA0101C0FB0109944E
:10344000CF93DF93C82FD62F0E94E1148C1740F042
:103450000E94E1148D1720F4DF91CF910C942F1965
:103460008C2FDF91CF910C943F191F93CF93DF9353
:10347000FB0112811111C3C0EC010E94DC0D8272AC
:10348000CD3CFCE5DF0709F49AC0A8F5C73CECE5A4
:10349000DE0709F476C0A8F4C43C9CE5D90709F41A
:1034A0005FC028F4C33CDC4509F457C054C0C53C98
:1034B0009CE5D90709F459C0C63CDC4509F45CC059
:1034C0004AC0CA3CFCE5DF0709F46AC050F4C83CB6
:1034D000ECE5DE0709F45AC0C93CDC4509F45BC0E1
:1034E0003AC0CB3C9CE5D90709F45FC0CC3CDC4535
:1034F00009F460C030C0C23DFCE5DF0709F46FC0CD
:1035000088F4CF3C9CE5D90709F460C008F45CC09E
:10351000C03DFCE5DF0709F45CC0C13DDC4509F4B2
:103520005BC019C0C53D9CE5D90709F460C050F4E3
:10353000C33DFCE5DF0709F455C0C43DDC4509F493
:1035400054C009C0C63D9CE5D90709F455C0CE3525
:10355000DD4509F454C011E052C00E944A194FC021
:103560004CE359E16FE279E104C04FE259E16CE3C9
:1035700079E10E941A1A43C04FE756E162E776E10B
:10358000F8CF42E756E16FE776E1F3CF4DE956E138
:103590006EE876E1EECF4EE856E16DE976E1E9CFEF
:1035A0004BEB56E16CEA76E1E4CF4CEA56E16BEB8B
:1035B00076E1DFCF44E155E16DEF74E1DACF4DEF15
:1035C00054E164E175E1D5CF81E017C065E082E0A8
:1035D00010C068E086E00DC06EE089E00AC064E1DA
:1035E0008FE007C067E185E104C088E106C062E2C0
:1035F00089E10E94201A03C083E20E943F19812FB3
:10360000DF91CF911F91089586E090E00C94D8252A
:10361000682F86E090E00C94EC258091D3028470B2
:1036200089618093D3020C94081B0E94C50E8111FE
:1036300004C00E946D0F0E940D1B0E94041B80930A
:10364000D302282F26952695269530E02430310583
:1036500024F0877088618093D3028091D30280FF29
:1036600004C086958695869501C080E00C94261C42
:103670002091D302822F869586958695482F50E01B
:103680004330510554F48F5F982F990F990F990F7C
:10369000822F8770892B8093D3028091D30281601F
:1036A0008093D3020E94081B8091D3028695869551
:1036B00086950C94261C8091D302982F969596950A
:1036C0009695A1F0915E990F990F990F8770892BAC
:1036D0008093D302887F91E009F490E08091D30237
:1036E00090FB80F98093D3020E94081B8091D30243
:1036F0008695869586950C94261C8091D30280FD34
:1037000013C081608093D302813019F489E08093E3
:10371000D3028091D3020E94081B8091D302869528
:10372000869586950C94261C08958091D30280FF7F
:1037300008C08E7F8093D3020E94081B80E00C9407
:10374000261C08958091D30280FD0C94951B0C9447
:103750007D1B9091D302892F8695869586958F5FE4
:103760008F719770843038F4880F880F880F892BF9
:103770008093D30202C09093D3028091D302887FBA
:1037800091E009F490E08091D30290FB80F980935E
:10379000D3020E94081B8091D30286958695869558
:1037A0000C94261C843008F083E09091D30297702B
:1037B000282F220F220F220F922B9093D302987F53
:1037C00021E009F420E09091D30220FB90F990933E
:1037D000D3020C94261C0E94D21B8091D3020C941D
:1037E000081B9C01FB018281882349F12E3BFCE5EB
:1037F0003F07C9F040F42C3BECE53E0769F02D3B58
:103800003C4561F00895203C9CE5390791F070F04B
:10381000213C3C4589F0089583E001C080E00E948E
:10382000EB1B80E008950E945B1BFBCF0E94381BBE
:10383000F8CF0E94A21BF5CF0E94A91BF2CF81E016
:1038400008958C9A94980895949808958F929F92D1
:10385000AF92BF92CF92DF92EF92FF920F931F939E
:10386000CF93DF93C82F843040F4811107C08FB508
:103870008F7D8FBD0E94241C04C0C3E08FB5806281
:103880008FBDA6B5B7B52C2F30E00E94892523E067
:1038900030E040E050E00E9459250027122F232FEE
:1038A000342F012F122F232F332786B597B56CE0C5
:1038B00070E00E9431256017710730F0C80169E09F
:1038C00070E00E94312552C086B597B5E6B4F7B4D2
:1038D000E6B5F7B5C6E0D0E0BE010E943125060F7F
:1038E000171F211D311D4801590185E0880C991CC5
:1038F000AA1CBB1C8A95D1F7C701BE010E943125C5
:103900006F01E12CF12CA7019601260F371F411DF5
:10391000511DC501B4010E94592569017A01E6B51E
:10392000F7B5CA01B9010E9413259B01AC01DF0163
:103930000E949F259B01AC01C701B6010E9413257F
:10394000DC01CB012FE0B695A795979587952A9531
:10395000D1F706B517B520E030E0081719072A0798
:103960003B0718F466B577B5CB01BC0179BD68BDDE
:10397000DF91CF911F910F91FF90EF90DF90CF904B
:10398000BF90AF909F908F90089508950E94211C42
:1039900082E28FBD89E18EBD8FEF9FEF97BD86BD1F
:1039A0000C94151B0F931F93CF93DF938C01EB01A6
:1039B0008091DA01811105C00E94162081E0809378
:1039C000DA01AE01440F551F4C0F5D1F24E630E0B5
:1039D000B80180EBDF91CF911F910F910C94C9201A
:1039E000CF93DF93EC01FB018281882309F43CC172
:1039F000C430FDE5DF0760F4CB3F9CE5D90788F4D0
:103A00009E0122503C452431310508F02EC109C0E9
:103A1000C236EDE5DE0729F0C63AFDE5DF0709F01D
:103A200024C10E94D80E90937F0280937E02C13100
:103A30008CE5D80709F4C6C008F042C0C930ECE5EF
:103A4000DE0709F49BC000F5C5308CE5D80709F402
:103A500085C078F4C330ECE5DE0709F478C008F0DF
:103A60007AC0C230DC4509F0F5C080917E028160E9
:103A7000EFC0C7309CE5D90709F478C008F07AC0D8
:103A800080917E028061E4C0CD30FCE5DF0709F45F
:103A900087C058F4CB309CE5D90709F479C008F009
:103AA0007BC080917E0288606FC0CF30FCE5DF076D
:103AB00009F480C008F082C080917E02877FC8C070
:103AC000CE3F9CE5D90709F471C000F5C531FCE58E
:103AD000DF0709F485C068F4C3319CE5D90709F410
:103AE00075C008F095C00E94890880917E028F778A
:103AF000AFC0CC3FFCE5DF07A9F108F054C0CB3FD5
:103B0000DC4509F0A7C080917F0240C0C230EDE5DE
:103B1000DE0709F489C058F4C1158DE5D80709F40A
:103B20005AC008F069C080917F0282602FC0C236FF
:103B3000EDE5DE0709F47CC0C63AFDE5DF0709F4D0
:103B400081C0C330DD4509F085C080E06EC0809142
:103B50007E0282607DC080917E0216C080917E02CE
:103B6000886076C080917F0282604FC080917E0223
:103B700080626EC080917E0280646AC00E94890863
:103B800080917E02806864C0846062C081603DC0B4
:103B900080917E028E7F5CC080917E028D7F58C0B6
:103BA00080917E0216C080917F0218C080917F02B2
:103BB0008D7F2BC080917E028F7E4AC080917E02D5
:103BC0008F7D46C080917E028F7B42C080917E02B5
:103BD000877F8B7F3DC080917F028D7F8E7F15C058
:103BE00080917E0282FB222720F991E0922790FBB0
:103BF00082F990FB83F92CC080917F02982F9095D9
:103C000091708E7F892B90FB81F980937F0222C077
:103C10000E94890880917E0287FB222720F991E08B
:103C2000922790FB87F914C081E00E946F0F12C0A9
:103C300080917E0284FB222720F991E0922790FB5D
:103C400084F906C080917E02982F909590FB80F9B0
:103C500080937E0280917E0290917F020E94E90E05
:103C60000E94890880E001C081E0DF91CF91089532
:103C70000F931F9341E050E060E070E08A019B01E8
:103C800004C0000F111F221F331F8A95D2F7C901EC
:103C9000B8010E94E1081F910F910C9489088B31A3
:103CA00009F468C058F58B3009F486C078F4863082
:103CB00009F445C020F4853009F44BC07FC087303B
:103CC00009F44AC0883009F477C078C0803109F41B
:103CD00064C068F48E3009F071C08091CA0182FB23
:103CE000222720F991E0922790FB82F94CC086317F
:103CF00009F462C0893109F45FC060C08A32E1F022
:103D000060F4873209F455C028F48E3108F456C0A7
:103D10008D5150C08932E9F051C0833450F48A3358
:103D200008F045C0853309F444C0883309F444C021
:103D300045C08334F1F142C00E946D0F3DC08091B7
:103D4000CA01817F8E7F8093CA0181E08093DB016D
:103D500008950E944C0430C08091CA01982F90951C
:103D6000917090FB80F98093CA01911125C0897FE1
:103D7000877F10C08091CA0181FB222720F991E042
:103D8000922790FB81F98093CA019923A9F0809131
:103D9000CA0181608093CA010FC08091CA0183FB70
:103DA000222720F991E0922790FB83F9ECCF8953E9
:103DB00001C080E00E94381E81E0089580E00895EF
:103DC00080E008950C94E01ECF93C82F8091DB0112
:103DD000882319F0813031F02BC00E94DC0D823233
:103DE00049F504C00E94DC0D823261F48C2F0E94E0
:103DF000E21E811104C08C2F0E944F1E17C081E06B
:103E000090E014C08C2F0E94E01E81110EC0C431BE
:103E100049F018F4CB3049F00FC0C93219F0C8335B
:103E200021F00AC01092DB0107C081E0817006C05A
:103E30001092DB0180E002C080E0F8CFCF910895BE
:103E4000CF93DF9386319C4541F5EB010E94DC0D59
:103E5000982F8A812091620030916300882379F045
:103E60009A7A81E009F480E08093DC01911102C02C
:103E700069E201C065E3C9010E947E210AC0809108
:103E8000DC01811102C069E201C065E3C9010E9441
:103E900080210E941E0E80E001C081E0DF91CF9161
:103EA00008950F931F93CF93DF93C42FD22FFC015C
:103EB00082818823C9F04093DF010E94BB21909347
:103EC000DE018093DD0180E28C0F883008F057C05E
:103ED000C77081E001C0880FCA95EAF7DF91CF91E2
:103EE0001F910F910C94F5058091DF01481330C0AC
:103EF0008091DD019091DE010E94D321883C9105E3
:103F000038F510E21D0FCD17B9F080E28C0F883024
:103F100040F4C77081E001C0880FCA95EAF70E949B
:103F2000FC05183028F581E09D2F977001C0880F9F
:103F30009A95EAF70E94F505802F0E94EC0518304B
:103F4000F0F4D77081E001C0880FDA95EAF70AC073
:103F500080E28C0F883098F4C77081E001C0880F30
:103F6000CA95EAF7DF91CF911F910F910C94FC0550
:103F7000802FDF91CF911F910F910C94EC05DF9171
:103F8000CF911F910F9108950F939C01CB01243F76
:103F90004CE5340731F188F4293DFCE53F07D9F0C1
:103FA0002A3D4CE5340779F1283D3C45A9F506E268
:103FB00021EE41EE68ED7CE52BC0263FFCE53F0796
:103FC000E1F0A8F0273F3C4539F507E225EE46EE43
:103FD00067EF7CE51DC007E225EE45EE69ED7CE567
:103FE00017C006E221EE40EE64EF7CE511C007E267
:103FF00025EE44EE65EF7CE50BC006E221EE42EED5
:1040000066EF7CE505C008E221E045EE6AED7CE55F
:104010000E94511F80E008C0FC018281882319F0B2
:104020001092DF0101C081E00F91089511B887E07F
:1040300080B985B3836085BB86B7846086BF86B749
:10404000816086BF86B7806486BF08959F92AF92D5
:10405000BF92CF92DF92EF92FF920F931F93CF9375
:10406000DF93B82EEB010E94BB216C01C431D10556
:1040700058F0CF3F8FEFD80759F0CE0164E170E0E0
:104080000E9431257B0107C0EE24E394F12C03C08C
:1040900025E0E22EF12C84E8A82E94EA992E16BE93
:1040A00096BE0E94BB218C0106B607FC08C00E9488
:1040B000BB21801B910B8E159F05B0F324C081B1ED
:1040C000887F883039F081B1887F803119F00FEF17
:1040D0001FEF1BC0B3B8A6BE0E94BB218C0106B661
:1040E00007FC08C00E94BB21801B910B8E159F0509
:1040F000B0F309C081B1887F883111F0803439F77D
:1041000000E010E00DC00EEF1FEFCF3F8FEFD8079C
:1041100031F2C6010E94D3218C179D0708F4BFCF4E
:10412000C801DF91CF911F910F91FF90EF90DF9029
:10413000CF90BF90AF909F9008950F931F93CF9310
:10414000DF93EB0183B984E886BF0E94BB218C0119
:1041500006B607FC0EC0CF3F8FEFD807C9F30E9409
:10416000BB21801B910B8C179D0790F38EEF9FEF67
:104170000BC021B1287F81E090E0283211F480E06B
:1041800090E0919581959109DF91CF911F910F91C9
:104190000895CF92DF92EF92FF920F931F93CF93E8
:1041A000DF936B018A017901B9010E942620E601A3
:1041B0000C0D1D1DC017D10759F424E926BFDF914E
:1041C000CF911F910F91FF90EF90DF90CF900895C6
:1041D00097FDF3CFB70189910E949D20EBCF90937B
:1041E00023018093220108959093E5018093E401D7
:1041F0000895E091E401F091E501309721F00190FC
:10420000F081E02D099480E00895E091E401F091BF
:10421000E501309721F00280F381E02D09940895A3
:104220002091E2013091E3012817390771F0909352
:10423000E3018093E201E091E401F091E501309720
:1042400021F00680F781E02D099408952091E00186
:104250003091E1012817390771F09093E1018093C3
:10426000E001E091E401F091E501309721F0008454
:10427000F185E02D09940895FC01329697E080E0E5
:10428000915029F021912223D9F38F5FF9CF08951E
:10429000662349F0FC01329608962191621729F0B5
:1042A000E817F907D1F780E0089581E008959C01AF
:1042B000FC0132969FEF80E04191461789F09F3FC5
:1042C00019F4411101C0982F8F5F8630A9F79F3FE5
:1042D00039F0F901E90FF11D97FDFA956283089510
:1042E00008959C012A5F3F4FFC014281461301C0A3
:1042F0001282019682179307B9F708950C945721FB
:104300000C947121029626E0FC0111922A95E9F79E
:10431000089508950C9489210C948A210C94892184
:104320000C9489210C948921CF930E9490210E94A2
:104330006A130E948E21C0E08C2F0E949412892B58
:1043400029F4CF5FC630C1F780E001C081E0CF9192
:10435000089508958091E80181110C94BB0408959B
:104360000E9489080C94C2048BE083BF8BEB8CBF46
:1043700082E089BF08952FB7F8948091D40290917C
:10438000D502A091D602B091D7022FBF08952FB7C2
:10439000F8946091D4027091D5028091D6029091E8
:1043A000D7022FBF08959C014FB7F8948091D40293
:1043B0009091D502A091D602B091D7024FBF821B37
:1043C000930B089578941F920F920FB60F921124B9
:1043D0008F939F93AF93BF938091D4029091D50216
:1043E000A091D602B091D7020196A11DB11D809374
:1043F000D4029093D502A093D602B093D702BF9176
:10440000AF919F918F910F900FBE0F901F901895B5
:1044100060E081E090E00E940F269CE088E10FB60A
:10442000F894A89581BD0FBE91BDFFCF0E94BB211E
:104430009093E7018093E60108950E94F8248B9AF7
:1044400080E0815041F0A895E7EBFBE03197F1F770
:1044500000C00000F6CF8B98789408950E941B232B
:104460000E94F4202FEB84ED91E021508040904099
:10447000E1F700C0000008958091FF02882389F0D1
:104480001092FF020E94BB219093E7018093E60106
:104490008091E8018823D1F11092E8010E94B021B7
:1044A00011C08091E801811111C08091E6019091C5
:1044B000E7010E94D321069728F081E08093E8016C
:1044C0000E94AA218091E801882301F10E94AA217B
:1044D0000E949421882339F1F89421B3939A822F72
:1044E0008C6081BB92B38CE0982792BB3FE54AEE8B
:1044F00090E0315040409040E1F700C0000092B39E
:10450000892782BB21BB9398789408950E94012447
:1045100080910503882329F08091E30284FD0E94A5
:104520005A100C94C222089580917D020895089536
:104530009091EE01981307C02091EC013091ED01AC
:1045400026173707A9F08093EE017093ED01609371
:10455000EC018093E9017093EB016093EA01809193
:104560001C0384FF05C063E089EE91E00C94FD23F9
:104570000895BC0184E00C949822BC0183E00C9463
:1045800098220895CF93DF93CAE0D0E08091E302B0
:1045900084FF18C08091FA019091FB019817E1F017
:1045A00028E0829FC001112468E084509E4F0E9441
:1045B000F9238091FA0190E001968F7099278093FA
:1045C000FA010AC00E94012487EB9BE00197F1F7F2
:1045D00000C000002197D1F6DF91CF910895CF93CD
:1045E000DF93EC01A091FB01B0E0CD0101968F704B
:1045F00099272091FA01281779F093E0AA0FBB1FA1
:104600009A95E1F7A450BE4F98E0FE0101900D92FB
:104610009A95E1F78093FB010E9401240E94C22237
:1046200088E0FE01A2EFB1E001900D928A95E1F7DA
:10463000DF91CF91089587E790E00895FC01808194
:1046400080768032A1F58181813061F48481958109
:10465000892B69F582EF91E0909301038093000329
:1046600088E00895823041F48CE792E09093010352
:104670008093000381E008958A3021F48381809340
:104680007C0215C0893099F4828193818115924012
:1046900081F484819581892B61F481E08093F1011B
:1046A000868197819093F0018093EF0102C080E0B2
:1046B00008958FEF08952091EF013091F001232BA1
:1046C00071F02091F101213051F4FC01808180933F
:1046D0007D021092F0011092EF0181E008958FEFBA
:1046E00008950895FC0193819330D9F068F49130D6
:1046F00081F0923009F059C08BEE93E09093010362
:10470000809300038BE30895913249F19232B9F11D
:104710004CC086E294E0909301038093000382E111
:1047200008958281813099F050F08230F1F588E36C
:1047300094E090930103809300038CE0089580E55A
:1047400094E0909301038093000384E0089586E44D
:1047500094E0909301038093000388E008958281A0
:10476000882329F0813009F586E194E002C08DEFBD
:1047700093E0909301038093000389E0089584817E
:104780009581009751F0019781F484E594E090932E
:1047900001038093000382E3089586E894E09093F8
:1047A00001038093000380E4089580E008951F933F
:1047B000CF93DF93162FEA01288124FF05C03981AA
:1047C00028E82327298302C02AE52883212FFC011A
:1047D000CE010296DC0131913D9321501216DCF39B
:1047E000612F0E9497021C5F1883DF91CF911F9168
:1047F000089543EE52E00C94D7234CE153E00C941F
:10480000D723CF93DF9360910203635067FD93C07A
:104810008091FE02CCE0D0E0C81BD109CA5FDC4F1A
:104820008091FD02803120F4CE010E94712381C06D
:104830008D3209F06EC0683009F07BC083EC809344
:10484000D8028AE5809384001092FC0288818076E9
:1048500021F0CE010E941E2349C09A811092E102EC
:104860008981811106C01092E20221EE32E082E0DD
:1048700038C0853019F49093030330C08630A1F41A
:104880008B81813041F0823031F0833021F08132F0
:1048900011F0823221F4CE010E94722301C080E027
:1048A00090E49093FC0222C0883089F0893019F49A
:1048B0009093050313C08A3069F08B3079F48BE450
:1048C0008093E40280931D038093F00207C025E0EB
:1048D00033E002C021EE32E081E003C021EE32E09D
:1048E00080E0309301032093000309C08F3F39F427
:1048F000988197FD8E8190E89093FC0207C09F817C
:10490000911104C09E81981708F4892F8093830029
:1049100010C08091FC0287FF0CC0CE010E945B2377
:104920008F3F21F48EE18093840003C081111092A7
:104930008300109202038091840084FF4CC0809118
:1049400083008F3F09F447C0C82F893008F0C8E0C2
:104950008C1B809383009091D80288E889278093EC
:10496000D802CC2359F1809100039091010320914A
:10497000FC0226FF12C0A8EDB2E02C2FAC01485D6E
:104980005240FA01EA0FFB1FE4911196EC93119744
:10499000215011962111F5CF08C0E9EDF2E0DC01BC
:1049A0002C2F3D9131932150E1F701962FEF2C0FE1
:1049B000820F911D90930103809300036C2F89ED6A
:1049C00092E00E949702CC5FCC3019F08FEF809379
:1049D0008300C093840084E190B39C7031F48150D3
:1049E000D9F7109203031092FB02DF91CF91089543
:1049F000CF93DF9385B7886085BF8BB780688BBF07
:104A0000C3EED2E08BE48983ACE1B3E011968C93E2
:104A10001197EFEEF2E081838AE588838C9380839F
:104A2000DF91CF910895DB018F939F930E949F2583
:104A3000BF91AF91A29F800D911DA39F900DB29F3A
:104A4000900D1124089587FB082E062687FD819579
:104A500067FD61950E94B2250EF4919507FC819542
:104A60000895AA1BBB1B51E107C0AA1FBB1FA617B5
:104A7000B70710F0A61BB70B881F991F5A95A9F707
:104A800080959095BC01CD01089597FB072E16F4F3
:104A9000009407D077FD09D00E94312507FC05D08E
:104AA0003EF4909581959F4F0895709561957F4F45
:104AB0000895A1E21A2EAA1BBB1BFD010DC0AA1F5F
:104AC000BB1FEE1FFF1FA217B307E407F50720F077
:104AD000A21BB30BE40BF50B661F771F881F991FF2
:104AE0001A9469F760957095809590959B01AC013B
:104AF000BD01CF010895EE0FFF1F0590F491E02D49
:104B000009940E948925332312F48A1B9B0B0C9471
:104B10009A25A29FB001B39FC001A39F700D811D74
:104B20001124911DB29F700D811D1124911D0895B6
:104B30000E948925B7FF0895821B930B08950E9458
:104B40008925A59F900DB49F900DA49F800D911D68
:104B500011240895B7FF0C949F250E949F25821B66
:104B6000930B0895991B79E004C0991F961708F0DC
:104B7000961B881F7A95C9F780950895FC014150CE
:104B8000504030F001900616D1F73197CF010895CB
:104B9000882799270895FB01DC0104C08D910190BD
:104BA000801921F441505040C8F7881B990B089593
:104BB000E199FECF9FBB8EBBE09A99278DB30895F4
:104BC000A6E1B0E044E050E00C941E26A8E1B0E07D
:104BD00042E050E00C941E26262FE199FECF9FBBA9
:104BE0008EBBE09A01970DB2021631F02DBB0FB6C5
:104BF000F894E29AE19A0FBE08950396272F0E9437
:104C0000ED250E94EC25252F0E94ED25242F0C94E4
:104C1000ED250196272F0E94ED250C94EC25262FDB
:104C2000E199FECF9FBB8EBB2DBB0FB6F894E29AE5
:104C3000E19A0FBE01960895DC01CB01FC01E199D8
:104C4000FECF06C0FFBBEEBBE09A31960DB20D92CF
:0C4C500041505040B8F70895F894FFCF91
:104C5C00C800AC01010102001200121201191A1B4A
:104C6C001C1D1E1F2021229422EF22C122BD22B91D
:104C7C00229722FF5AE200E900EA00B500B600B71D
:104C8C0000CD008301CC008A019201940121022302
:104C9C000224022502260227022A02B300B4006F66
:104CAC00007000818283E200E900EA00B500B600E2
:104CBC00B700CD008301CC008A019201940121023E
:104CCC00230224022502260227022A02B300B40082
:104CDC006F00700081828390919293949596973790
:104CEC003635343332076061626364650001020259
:104CFC0002020606060909090909090F0F0F0F0F11
:104D0C000F15151518191919191919191919192314
:024D1C00240071
:00000001FF
